:0400000006EF00F017
:10000800E1EF1CF000EE70F0900EEE6AE806FDE1FC
:10001800076A07EE4EF017EE2CF0EE6AE550E15055
:10002800FCE1E250FAE107EE3CF0580EF66E000EE5
:10003800F76EF86A10EE12F00900F5CFEEFFE55002
:10004800E150FAE1E25002E020EF00F03CEF1FF04F
:10005800C0A80296C0A80264C0A802FF0036374AAA
:100068003630FE00FEC0F6FFFFC0F7FF0E0EF76445
:1000780003D00800F55005D0F6CFE9FFF7CFEAFF27
:10008800EF501200EC000001FA6BFB6BECC0F8F0CB
:10009800EDC0F9F00001F051FE6FF151FF6FF04B28
:1000A800F12BE0DF0001F56FF55101E176D2F55152
:1000B800250A0AE0FA4BFB2BEF51EE1101E068D15B
:1000C800F551C1EC1CF0E6D70001F269F46BF36B53
:1000D8001ED20001EF51EE1106E0EEC0E9FFEFC0BD
:1000E800EAFF000EEF6AFAC000F0FBC001F0120050
:1000F800F8C0E9FFF9C0EAFF0001020EF827000E78
:10010800F923EF503DD20001F38D01D2100E05D036
:10011800080E03D00001F32B0A0E0001F26FF8C09D
:10012800E9FFF9C0EAFF020EF827000EF923EECF27
:10013800F6F0EDCFF7F0F3A10DD0F7AF06D0F66DDE
:10014800F71FD8B0F72BF40707D00001F391F3ADF0
:1001580003D0F9D70001F391F2C002F0036AF6C0A8
:1001680000F0F7C001F0E0EC02F000500001F56F7C
:10017800F2C002F0036AF6C000F0F7C001F0E0EC4C
:1001880002F004C0F6F005C0F7F0010EFC6FFD6B3D
:100198000001FD51F75D02E1FC51F65D12E3F2C08A
:1001A80002F0036AFCC000F0FDC001F013EC03F09C
:1001B80004C0FCF005C0FDF00001F451E9E0F407CB
:1001C800E7D70001F3A913D018D00001FA4BFB2B95
:1001D800EF51EE1109E0EEC0E9FFEFC0EAFF200E93
:1001E800EF6EEE4BEF2B03D0200EC1EC1CF000019C
:1001F800F407F451800A7F0FE8E20001F3A112D05E
:10020800FA4BFB2BEF51EE1109E0EEC0E9FFEFC00E
:10021800EAFF2D0EEF6EEE4BEF2B15D02D0EC1EC35
:100228001CF011D00001F3AD0ED0FA4BFB2BEF51AF
:10023800EE1106E0EEC0E9FFEFC0EAFF2B0EEAD7A9
:100248002B0EC1EC1CF00001F3B913D04AD0000109
:10025800FA4BFB2BEF51EE1109E0EEC0E9FFEFC0BE
:10026800EAFF300EEF6EEE4BEF2B03D0300EC1ECF1
:100278001CF00001F407F451800A7F0F32E3E7D73E
:10028800FCC002F0FDC003F0F6C000F0F7C001F0BA
:10029800E0EC02F004C000F005C001F0F2C002F08A
:1002A800036AE0EC02F000500001F46FF451800A98
:1002B800760F02E3070EF4270001FA4BFB2BEF51F0
:1002C800EE110AE0F451300FEEC0E9FFEFC0EAFF8B
:1002D800EF6EEE4BEF2B05D00001F451300FC1EC5F
:1002E8001CF0F2C002F0036AFC0EE96E000EEA6E22
:1002F800EE50006EEF50016EE0EC02F00550ED6E2E
:100308000450EF6EEE50ED10BBE1090E0001F565EB
:1003180002D0070EF5270001FA4BFB2BEF51EE1127
:1003280008E0F551300FEEC0E9FFEFC0EAFFEF6ECD
:1003380035D00001F551300FC1EC1CF0ABD60001EF
:10034800F451800A7E0F14E3FA4BFB2BEF51EE11A8
:1003580009E0EEC0E9FFEFC0EAFF200EEF6EEE4BBA
:10036800EF2B03D0200EC1EC1CF00001F407E7D7F7
:10037800F8C0E9FFF9C0EAFF0001020EF827000EF5
:10038800F923EF50F56FFA4BFB2BEF51EE1109E013
:10039800EEC0E9FFEFC0EAFFF5C0EFFFEE4BEF2B31
:1003A80079D60001F551C1EC1CF074D6F8C0E9FF0C
:1003B800F9C0EAFF0001020EF827000EF923EECF7C
:1003C80000F0EDCF01F000C070F001C071F0D96A03
:1003D80070C000F071C001F0D9500024026E000E08
:1003E8000120036E02C0F6FF03C0F7FF0E0EF7648C
:1003F80003D00800F55005D0F6CFE9FFF7CFEAFFA4
:10040800EF50000902E0D92AE3D70001F251D96080
:1004180002D0D950F26F0001F251F4BF3BD0FF0A6D
:10042800F425000138E3FA4BFB2BEF51EE1109E0FC
:10043800EEC0E9FFEFC0EAFF200EEF6EEE4BEF2BA8
:1004480003D0200EC1EC1CF00001F407E4D7000132
:1004580070C000F071C001F00028706F02E101283F
:10046800716F00C0FEF001C0FFF0FCDD0001F56F08
:10047800FA4BFB2BEF51EE1109E0EEC0E9FFEFC09C
:10048800EAFFF5C0EFFFEE4BEF2B04D00001F5516A
:10049800C1EC1CF00001F207F22901E1FBD5D7D726
:1004A800F0C0FEF0F1C0FFF0DDDD2A0A0EE1F8C071
:1004B800E9FFF9C0EAFF0001020EF827000EF92350
:1004C800EF50F26FF04BF12B22D00001F051FE6F8C
:1004D800F151FF6FF04BF12BC5DDD00F0001F26F2A
:1004E800F0C0FEF0F1C0FFF0BDDDD96E2F0ED9646B
:1004F8000ED03A0ED9600BD00001F2510A0DD95036
:10050800F324D00FDED70001F3B52DD0F389000115
:10051800F051FE6FF151FF6FF04BF12BA3DD00019D
:10052800F56FF55101E1D5D52A0A01E1E1D5010AB6
:1005380001E1E9D5050AB4E01E0AE5E0680A01E12F
:10054800E5D53B0A01E1FBD6070A01E1E3D50B0A31
:1005580001E1DED51C0A01E129D7060A01E1DCD553
:100568000D0A01E1D3D52F0E0001F5650BD03A0E27
:10057800F56108D0F385F4510A0DF551F324D00F35
:10058800F46FC5D70001FA4BFB2BEF51EE1101E0D8
:10059800FFD6F551C1EC1CF07DD50001EF51EE11ED
:1005A80006E0EEC0E9FFEFC0EAFF000EEF6AFAC00E
:1005B80000F0FBC001F01200066A046A056A0250E6
:1005C800031003E1006A016A000C1F0E0612D8909E
:1005D800062A02360336FCE3033202320250005C7C
:1005E8000350015804E3016E0250005ED8800436BF
:1005F8000536062E06BAF0D706AE05D0041E042A24
:10060800D8B40506051E0450026E0550036E06ACEC
:10061800000C001E002AD8B40106011E000C02506E
:100628000002F3CF04F0F4CF05F002500102F350BA
:10063800052603500002F35005261200EEC0F0F024
:10064800EFC0F1F0000EE8CFEEF0E8CFEFF047EFA3
:1006580000F0046E042A0406D8B4000CD8900332C3
:10066800023201320032F7D7046E042A0406D8B4E5
:0E067800000CD8900036013602360336F7D754
:100F00000D0A454454502036374A36302044726921
:100F10007665723E0031384636374A3630204472A4
:100F200069766572000D0A4D59204D4143204144B8
:100F30004452455353203D2030302D30302D34362F
:100F40002D35342D34392D3439004D41433A30306C
:100F50003030343635343439313900495020414449
:100F60004452455353000D0A4E45572049502041E5
:100F7000444452455353203D200047415445574176
:100F8000592049502041444452455353000D0A4EC4
:100F90004557204741544557415920495020414425
:100FA0004452455353203D20005355424E45542052
:100FB0004D41534B000D0A4E4557205355424E4567
:100FC00054204D41534B203D200020202044454DCE
:100FD0004F20424F415244000D0A41525020526569
:100FE000706C79205472616E736D697373696F6E82
:100FF0002041626F727465642E2E000D0A554450B4
:1010000020446174616772616D205472616E736D0A
:10101000697373696F6E2041626F727465642E2EFE
:10102000000D0A544350205472616E736D697373DE
:10103000696F6E2041626F727465642E2E000D0A16
:101040004E45572047415445574159204144445249
:101050004553532049532025642E25642E25642EA4
:1010600025642E2E000D0A4E45572049502041443C
:1010700044524553532049532025642E25642E2580
:10108000642E25642E2E000D0A4E455720535542DE
:101090004E4554204D41534B2049532025642E2565
:1010A000642E25642E25642E2E000D0A44484350DC
:1010B00020494E49542E2E000D0A444843502052D8
:1010C000455345542E2E000D0A53454E5420444896
:1010D00043502052455155455354204D455353419B
:1010E00047452E2E000D0A53454E54204449534384
:1010F0004F564552204D4553534147452E2E000D26
:101100000A52454345495645442044484350204FE0
:1011100046464552204D4553534147452E2E000D1E
:101120000A524543454956454420444843502041CE
:10113000434B204D4553534147452E2E000D0A5237
:10114000454345495645442044484350204E414B71
:10115000204D4553534147452E2E000D0A44484328
:1011600050204C454153452054494D452045585049
:10117000495245442E2E002036374A3630204554F9
:101180004845524E455420000D0A36374A36302025
:10119000496E697469616C697A65640D0A00E96E6B
:1011A000E906E928D8B41200040EE16EE106E12850
:1011B000F7E0770ED96E02D000F000F0D92EFCD700
:1011C000F5D7D96ED950040AD8A41200966A956A48
:1011D00016D8020E2DD81FD8020E2AD81CD8080EF9
:1011E00027D819D8000E24D816D80E0E21D813D817
:1011F000000E1ED810D8060E1BD80DD82FD0030E07
:101200000001D96F0001D951D8B41200846A03D803
:101210000001D907F7D7020EC2DF83928380320E16
:10122000D96E02D000F000F0D92EFCD783901200C6
:10123000D96ED944E846FC0B846E320ED96E02D0CA
:1012400000F000F0D92EFCD71200F36EF38EF338C5
:101250000F0BEEDFE0DFF350EBDFDDD7010EE8DF51
:10126000DADF000EE5DFD7D7E600F46EF450EDDFED
:10127000320ED96E02D000F000F0D92EFCD7838256
:10128000E6C0F6FFE7C0F7FF0E0EF76403D00800D4
:10129000F55005D0F6CFE9FFF7CFEAFFEF50000990
:1012A000D8B41200E6C0F6FFE7C0F7FF0E0EF764F1
:1012B00003D00800F55005D0F6CFE9FFF7CFEAFFDD
:1012C000EF50006E00380F0BB3DF83800A0ED96E2B
:1012D00002D000F000F0D92EFCD78390E6C0F6FFD4
:1012E000E7C0F7FF0E0EF76403D00800F55005D0F5
:1012F000F6CFE9FFF7CFEAFFEF509ADF83800A0EBF
:10130000D96E02D000F000F0D92EFCD783900001F6
:10131000E64BE72BB5D7D96EE16AE15007EE6DF0E9
:10132000E926000EEA22300EEF6EE12A020EE16499
:10133000F4D7D9CF00F0016A0150800A7F0F000E68
:10134000D8B4005CD8B01200630ED96407D09C0EEC
:10135000D92607016D2B640ED960F9D7090ED9641F
:1013600007D0F60ED92607016E2B0A0ED960F9D7E1
:10137000D95007016F27120000EE98F0EE6AEE6A6E
:101380000A0EE8CFE2FE1A0EE8CFE3FE060EF36E79
:10139000F46AF350006EF450016EF306000EF45A36
:1013A0000150001004E0FF0EE8CFFAFEF2D7480E1D
:1013B000E16E070EE26E060EF36EF46AF350006EF5
:1013C000F450016EF306000EF45A0150001003E0D1
:1013D000E6CFFAFEF3D7080EE8CFFAFE0E01FA6B5D
:1013E00000010F0E9827000E9923450EE8CFFAFE54
:1013F0000E01FA6BFA6BFA6BFA6B010EE8CFFAFE8C
:10140000FA6BFA6B640EE8CFFAFE110EE8CFFAFE23
:10141000FA6BFA6B040EF36EF46A3C0EE16E070E83
:10142000E26EF350006EF450016EF306000EF45AB3
:101430000150001003E0E6CFFAFEF3D7040EF36E7E
:10144000F46A440EE16E070EE26EF350006EF45043
:10145000016EF306000EF45A0150001003E0E6CFCF
:10146000FAFEF3D70001140E9827000E99231F0EE1
:10147000E8CFFAFE980EE8CFFAFE760EE8CFFAFE35
:101480005F0EE8CFFAFE0E01FA6BFA6BFA6BFA6B9D
:101490000001080E9827000E9923240EF36EF46ABB
:1014A000240E9827000E9923250E846F0F0E856F4A
:1014B000F350006EF450016EF306000EF45A015022
:1014C000001016E084C0F6FF85C0F7FF0E0EF7642B
:1014D00003D00800F55005D0F6CFE9FFF7CFEAFFBB
:1014E000EF50E8CFFAFE0001842B000E8523E0D7F1
:1014F000130EF36EF46A0001130E9827000E992361
:10150000660E846F0F0E856FF350006EF450016EFF
:10151000F306000EF45A0150001016E084C0F6FFE6
:1015200085C0F7FF0E0EF76403D00800F55005D014
:10153000F6CFE9FFF7CFEAFFEF50E8CFFAFE000160
:10154000842B000E8523E0D7F66AF76A07EE3CF09D
:10155000F650E926F750EA22EF50DDDE6D0EE16E1F
:10156000070EE26E030EF36EF46A0001030E982775
:10157000000E99236DC7E8FF300A07E19807000EB7
:10158000995BF306D8A0F406E6526EC7E8FF300A6E
:101590000CE16DC7E8FF300A08E100019807000E72
:1015A000995BF306D8A0F406E652F350006EF450AF
:1015B000016EF306000EF45A0150001003E0E6CF6E
:1015C000FAFEF3D7000EF75C030ED8B4F65C07E220
:1015D0002E0EE8CFFAFE0001982B000E9923F64A52
:1015E000F72A000EF75C040ED8B4F65CAFE31B0ECE
:1015F000F36EF46A00011B0E9827000E99238D0EDE
:10160000846F0F0E856FF350006EF450016EF30679
:10161000000EF45A0150001016E084C0F6FF85C099
:10162000F7FF0E0EF76403D00800F55005D0F6CF93
:10163000E9FFF7CFEAFFEF50E8CFFAFE0001842B75
:10164000000E8523E0D7F66AF76A07EE70F0F650D1
:10165000E926F750EA22EF505EDE6D0EE16E070ECE
:10166000E26E030EF36EF46A0001030E9827000E7B
:1016700099236DC7E8FF300A07E19807000E995BD0
:10168000F306D8A0F406E6526EC7E8FF300A0CE174
:101690006DC7E8FF300A08E100019807000E995B6A
:1016A000F306D8A0F406E652F350006EF450016E33
:1016B000F306000EF45A0150001003E0E6CFFAFEE4
:1016C000F3D7000EF75C030ED8B4F65C07E22E0EDB
:1016D000E8CFFAFE0001982B000E9923F64AF72A6C
:1016E000000EF75C040ED8B4F65CAFE3140EF36E94
:1016F000F46A0001140E9827000E9923B50E846F2A
:101700000F0E856FF350006EF450016EF306000E5D
:10171000F45A0150001016E084C0F6FF85C0F7FFB0
:101720000E0EF76403D00800F55005D0F6CFE9FFA0
:10173000F7CFEAFFEF50E8CFFAFE0001842B000E4E
:101740008523E0D7F66AF76A07EE74F0F650E926CB
:10175000F750EA22EF50DFDD6D0EE16E070EE26E0C
:10176000030EF36EF46A0001030E9827000E99230E
:101770006DC7E8FF300A07E19807000E995BF30692
:10178000D8A0F406E6526EC7E8FF300A0CE16DC738
:10179000E8FF300A08E100019807000E995BF306A4
:1017A000D8A0F406E652F350006EF450016EF30632
:1017B000000EF45A0150001003E0E6CFFAFEF3D712
:1017C000000EF75C030ED8B4F65C07E22E0EE8CFED
:1017D000FAFE0001982B000E9923F64AF72A000E14
:1017E000F75C040ED8B4F65CAFE31B0EE8CFE2FE64
:1017F0001A0EE8CFE3FE98C000F099C001F0F10E98
:101800000024F36EFF0E0120F46EF4CFFAFEF3CF46
:10181000FAFE310EE8CFE2FE1A0EE8CFE3FE98C0E2
:1018200000F099C001F0DD0E0024F36EFF0E0120E0
:10183000F46EF4CFFAFE0001140E7E6F7F6B190E6A
:10184000886F1A0E896F88C0F0FE89C000F0016AA7
:1018500000C0F1FE7EC000F07FC001F0FF0E000668
:10186000012200C0E8FF882701C0E8FF892388C063
:10187000F2FE89C000F0016A00C0F3FE0E01300ED6
:10188000DF130E01DFBBFDD70001F6CE7AF07B6BD4
:10189000F7CE78F0796B230E886F1A0E896F88C0A7
:1018A000E2FE89C000F0016A00C0E3FE78C0FAFEE3
:1018B0007AC0FAFE090E98271A0E992398C0E6FE00
:1018C00099C000F0016A0050E8CFE7FE0E01FCA3CA
:1018D00004D00E01FC93DF87DF979E980E01DF870F
:1018E0000E01DFA71200FCD74EC7E8FF080AD8B4E4
:1018F000120007014E6B07015A6B120078D10001EC
:10190000B80EEE6F100EEF6F22EC03F0F36AF46A7C
:1019100007EE80F0F350E926F450EA22000EEF6A59
:10192000F34AF42AF45C040ED8B4F35CF1E3010E3C
:10193000E8CF4EF70001AA0EEE6F100EEF6F22EC0B
:1019400003F0F36AF46A07EE9CF0F350E926F450D2
:10195000EA22FF0EEF6EF34AF42A000EF45C060E44
:10196000D8B4F35CF0E3F36AF46A07EE78F0F3506E
:10197000E926F450EA22FF0EEF6EF34AF42A000E35
:10198000F45C040ED8B4F35CF0E300EE82F0EE6A8F
:10199000EE6A020EE8CF4EF70001070E835DD00E0F
:1019A000D8B4825DD8A01200030EE8CF4EF7120023
:1019B0000001B56BB46BB36B3C0EB26F07015AA15B
:1019C00004D0050EE8CF4EF71200010E2AD900EE22
:1019D00082F0EE6AEE6A040EE8CF4EF70001E50EE3
:1019E000EE6F100E3AEF1EF00001070E835DD00E71
:1019F000D8B4825D04E3030EE8CF4EF7120007016E
:101A00005AA91200DBDA020A0AE1050EE8CF4EF706
:101A10000001FF0EEE6F100EEF6F22EC03F00701D6
:101A20005A991200030EFDD800EE82F0EE6AEE6ABB
:101A3000060EE8CF4EF70001C70EEE6F100E3AEF1C
:101A40001EF007015AA905D0B9DAE8CF5CF7070103
:101A50005A995CC7E8FF060A08E100013D0EEE6FE7
:101A6000110EEF6F22EC03F03FD75CC7E8FF050AC9
:101A700001E093D000011F0EEE6F110EEF6F22EC0C
:101A800003F000EEAEF0EE6AEE6AEE6AEE6A070E62
:101A9000E8CF4EF7F36AF46A17EE80F0F350E126D0
:101AA000F450E22207EE3CF0F350E926F450EA222B
:101AB000E7CFEFFF17EE88F0F350E126F450E22273
:101AC00007EE74F0F350E926F450EA22E7CFEFFF77
:101AD00017EE7CF0F350E126F450E22207EE70F0AE
:101AE000F350E926F450EA22E7CFEFFFF34AF42A55
:101AF000000EF45C040ED8B4F35CCEE307015A8107
:101B00000001650EEE6F100EEF6F3FC7DFF0E06B68
:101B10003EC7DDF0DE6B3DC7DBF0DC6B3CC7D9F0C8
:101B2000DA6BD90EE8CFECF0000EE8CFEDF022EC46
:101B300003F000013E0EEE6F100EEF6F73C7DFF083
:101B4000E06B72C7DDF0DE6B71C7DBF0DC6B70C77A
:101B5000D9F0DA6BD90EE8CFECF0000EE8CFEDF05B
:101B600022EC03F00001870EEE6F100EEF6F77C7C7
:101B7000DFF0E06B76C7DDF0DE6B75C7DBF0DC6BAA
:101B800074C7D9F0DA6BD90EE8CFECF0000EE8CFCD
:101B9000EDF022EC03F0BCEF09F00001070E835DCD
:101BA000D00ED8B4825DD8A01200030EE8CF4EF755
:101BB000120000EEB2F00001EE52EE52EE52ED5085
:101BC000B15D08E1ED50B05D05E1ED50AF5D02E1C2
:101BD000EF50AE5DD8A0120000015B0EEE6F110E4B
:101BE000EF6F22EC03F0010EE8CF4EF712004EC764
:101BF000E8FF000A01E183D6010A01E19BD6030A4E
:101C000001E1CAD6010A01E1D3D6070A01E1ECD607
:101C1000010A01E107D7030A01E113D7010AC9E06C
:101C20001200D96E10EE98F0E66AE66A0A0EE8CF66
:101C3000E2FE1A0EE8CFE3FE0E0EE8CFFAFE060E25
:101C4000F36EF46AF450F31007E0FF0EE8CFFAFEEB
:101C5000F306D8A0F406F6D7480EE16E070EE26E42
:101C6000060EF36EF46AF450F31007E0E7CFFAFEC5
:101C7000E652F306D8A0F406F6D7080EE8CFFAFE2F
:101C80000E01FA6B00010F0E9827000E9923450EE6
:101C9000E8CFFAFE0E01FA6BFA6BFA6BFA6B010EE3
:101CA000E8CFFAFEFA6BFA6B640EE8CFFAFE110E7B
:101CB000E8CFFAFEFA6BFA6B040EF36EF46AF45096
:101CC000F31006E00E01FA6BF306D8A0F406F7D77E
:101CD000040EF36EF46AF450F31007E0FF0EE8CF41
:101CE000FAFEF306D8A0F406F6D70001140E9827E2
:101CF000000E99230E01FA6B440EE8CFFAFEFA6B40
:101D0000430EE8CFFAFEFA6BFA6BFA6BFA6B00013E
:101D1000080E9827000E9923010EE8CFFAFEE8CFAF
:101D2000FAFE060EE8CFFAFE0E01FA6B010EE8CFBE
:101D3000FAFE020EE8CFFAFE030EE8CFFAFE040E1A
:101D4000E8CFFAFEFA6BFA6B800EE8CFFAFEFA6B78
:101D5000100EF36EF46AF450F31006E00E01FA6B05
:101D6000F306D8A0F406F7D7480EE16E070EE26E30
:101D7000060EF36EF46AF450F31007E0E7CFFAFEB4
:101D8000E652F306D8A0F406F6D7CA0EF36EF46A4C
:101D9000F450F31006E00E01FA6BF306D8A0F40637
:101DA000F7D70001EC0E9827000E9923630EE8CFB9
:101DB000FAFE820EE8CFFAFE530EE8CFFAFE630E6B
:101DC000E8CFFAFE350EE8CFFAFE010EE8CFFAFEB4
:101DD000D9CFFAFE070E9827000E9923D90402E105
:101DE00007015A93D9042BE00701805328E017EE2E
:101DF00081F0E75024E017EE82F0E75020E017EE84
:101E000083F0E7501CE0360EE8CFFAFE040EE8CF70
:101E1000FAFE780EE16E070EE26E040EF36EF46ABF
:101E2000F450F31007E0E7CFFAFEE652F306D8A02D
:101E3000F406F6D70001060E9827000E9923370EF8
:101E4000E8CFFAFE020EE8CFFAFE010EE8CFFAFE66
:101E5000030EE8CFFAFE0001040E9827000E992326
:101E6000D950030A1CE1320EE8CFFAFE040EE8CF87
:101E7000FAFE800EE16E070EE26E040EF36EF46A57
:101E8000F450F31007E0E7CFFAFEE652F306D8A0CD
:101E9000F406F6D70001060E9827000E9923FF0ED0
:101EA000E8CFFAFE0001982B000E99231B0EE8CF15
:101EB000E2FE1A0EE8CFE3FE98C000F099C001F0F0
:101EC000F10E0024F36EFF0E0120F46EF4CFFAFE43
:101ED000F3CFFAFE310EE8CFE2FE1A0EE8CFE3FEB2
:101EE00098C000F099C001F0DD0E0024F36EFF0EE3
:101EF0000120F46EF4CFFAFEF3CFFAFE140E7E6FDB
:101F00007F6B190E886F1A0E896F88C0F0FE89C02A
:101F100000F0016A00C0F1FE7EC000F07FC001F059
:101F2000FF0E0006012200C0E8FF882701C0E8FF7D
:101F3000892388C0F2FE89C000F0016A00C0F3FE68
:101F40000E01300EDF130E01DFBBFDD70001F6CE10
:101F50007AF07B6BF7CE78F0796B230E886F1A0ED0
:101F6000896F88C0E2FE89C000F0016A00C0E3FE0C
:101F700078C0FAFE7AC0FAFE090E98271A0E992345
:101F800098C0E6FE99C000F0016A00C0E7FEFCCEF2
:101F9000D9FFD9CF00F0020E0016000404E10E01B3
:101FA000FC93DF87DF979E980E01DF87DFCE00F07E
:101FB000080E00160004D8A41200F8D70701686BB9
:101FC00007015A9546CAE8FF020A01E0CAD15AB38E
:101FD00018D0F36AF46A1AEE56F0F350E126F45082
:101FE000E22207EE80F0F350E926F450EA22E7CF30
:101FF000EFFFF34AF42A000EF45C040ED8B4F35C4D
:10200000EAE348C7E8FF0A016263ABD149C7E8FFCA
:102010000A016363A6D14AC7E8FF0A016463A1D13C
:102020004BC7E8FF0A0165639CD14CC7E8FF0A0172
:10203000666397D14DC7E8FF0A01676392D100013B
:10204000360E8C6F0B0E8D6F8CC0E9FF8DC0EAFFD2
:10205000EFCF5BF700018C2B000E8D236CD18CC071
:10206000E9FF8DC0EAFFEFCF67F700018C2B000E70
:102070008D2367C700F0000411E18CC0E9FF8DC01B
:10208000EAFFEFCF68F78C2B000E8D2307015AA3D0
:1020900065D168C7E8FF020A01E060D107015A87ED
:1020A0005DD18CC0E9FF8DC0EAFFEFCF67F700017B
:1020B0008C2B000E8D2367C7E8FF040AEFE1F36A5B
:1020C000F46A8CC0E9FF8DC0EAFF17EE8CF0F35084
:1020D000E126F450E222EFCFE7FF00018C2B000E47
:1020E0008D23F34AF42AF45C040ED8B4F35C01E3C4
:1020F00035D1E7D78CC0E9FF8DC0EAFFEFCF67F796
:1021000000018C2B000E8D2367C7E8FF040AC6E18F
:10211000F36AF46A8CC0E9FF8DC0EAFF17EE88F01D
:10212000F350E126F450E222EFCFE7FF00018C2BC1
:10213000000E8D23F34AF42AF45C040ED8B4F35C49
:1021400001E30CD1E7D78CC0E9FF8DC0EAFFEFCFE8
:1021500067F700018C2B000E8D2367C7E8FF040A88
:102160009DE10701F36A5AA30DD0F46A00018C2B9C
:10217000000E8D23F34AF42AF45C040ED8B4F35C09
:1021800019E2F4D7F46A8CC0E9FF8DC0EAFF17EEBC
:1021900084F0F350E126F450E222EFCFE7FF000194
:1021A0008C2B000E8D23F34AF42AF45C040ED8B471
:1021B000F35CE9E3080E84C700F0016A026A036A6F
:1021C00038EC03F000C0E1F001C0E2F002C0E3F03F
:1021D00003C0E4F085C700F0016A026A036A0001E7
:1021E000E1510026E2510122E3510222E45103228F
:1021F000080E38EC03F000C0E5F001C0E6F002C0C4
:10220000E7F003C0E8F086C700F0016A026A036ADB
:10221000E5510026E6510122E7510222E85103224E
:10222000080E38EC03F000C0E9F001C0EAF002C08B
:10223000EBF003C0ECF087C700F0E9510024E8CFD1
:10224000B2F0000EEA21E8CFB3F0000EEB21E8CFA8
:10225000B4F0000EEC21E8CFB5F000EEB5F0000EC2
:10226000ED5C08E1000EED5C05E1070EED5C02E1BE
:10227000090EEF5C73E30001F80EB227B323FF0EE3
:10228000B423B5236BD08CC0E9FF8DC0EAFFEFCF3C
:1022900067F700018C2B000E8D23030E0701676585
:1022A0002AD00701F36A5AA30DD0F46A00018C2BDF
:1022B000000E8D23F34AF42AF45C040ED8B4F35CC8
:1022C0001CE2F4D7F46A8CC0E9FF8DC0EAFF17EE78
:1022D0007CF0F350E126F450E222EFCFE7FF00015B
:1022E0008C2B000E8D23F34AF42AF45C040ED8B430
:1022F000F35CE9E302D007015A870701FC0E672768
:102300000701670767292AE000018C2B000E8D2347
:10231000F7D707015A8522D08CC0E9FF8DC0EAFFAC
:10232000EFCF67F700018C2B000E8D2307016707A5
:10233000672914E0F7D75BC7E8FF010A01E1DAD6A5
:10234000020AA1E0300A01E1FED6060A01E187D6C1
:10235000030A01E1A6D6C90ADCE0DED707015AA5C7
:1023600073D668C7E8FF020A1BE1F36AF46A17EE46
:102370008CF0F350E126F450E22207EE78F0F350AF
:10238000E926F450EA22E7CFEFFFF34AF42A000EE1
:10239000F45C040ED8B4F35CEAE307015A8316D068
:1023A00078C7E8FF07018C190FE179C7E8FF07013B
:1023B0008D190AE17AC7E8FF07018E1905E17BC78D
:1023C000E8FF07018F1902E00701686B07015AA7B0
:1023D00002D007015A9968C7E8FF120007015E970B
:1023E0000A0EF36E1A0EF46E0A0EE8CFE2FE1A0E13
:1023F000E8CFE3FE0E0EE8CFFAFEF34AF42AF66ABF
:10240000F76AFF0EE8CFFAFEF34AF42AF64AF72AF3
:10241000000EF75C060ED8B4F65CF3E3F66AF76AD2
:1024200007EE48F0F650E926F750EA22EFCFFAFE21
:10243000F34AF42AF64AF72A000EF75C060ED8B4DF
:10244000F65CEEE3080EE8CFFAFE060EE8CFFAFEE1
:10245000020EF326000EF4220E01FA6B010EE8CFF5
:10246000FAFE020EF326000EF422080EE8CFFAFE62
:10247000FA6B020EF326000EF422060EE8CFFAFEE7
:10248000040EE8CFFAFE020EF326000EF422FA6BD9
:10249000010EE8CFFAFE020EF326000EF422F66AD1
:1024A000F76A07EE48F0F650E926F750EA22EFCF38
:1024B000FAFEF34AF42AF64AF72A000EF75C060EF3
:1024C000D8B4F65CEEE3F66AF76A07EE3CF0F65035
:1024D000E926F750EA22EFCFFAFEF34AF42AF64A49
:1024E000F72A000EF75C040ED8B4F65CEEE3F66A49
:1024F000F76A0E01FA6BF34AF42AF64AF72A000E3D
:10250000F75C060ED8B4F65CF4E3F66AF76A07EEF9
:1025100040F0F650E926F750EA22EFCFFAFEF34AF0
:10252000F42AF64AF72A000EF75C040ED8B4F65CDB
:10253000EEE3F3CFE6FEF4CFE7FEDFCE00F0080EC9
:1025400000160004FAE00E01DF8712000A0EF36E97
:102550001A0EF46E0A0EE8CFE2FE1A0EE8CFE3FE82
:102560000E0EE8CFFAFEF34AF42AF66AF76A0AEE8C
:1025700022F0F650E926F750EA22EFCFFAFEF34AAE
:10258000F42AF64AF72A000EF75C060ED8B4F65C79
:10259000EEE3F66AF76A07EE48F0F650E926F750E0
:1025A000EA22EFCFFAFEF34AF42AF64AF72A000E9F
:1025B000F75C060ED8B4F65CEEE30001280E746FEB
:1025C0000A0E756F020EE8CF31FAF66AF76A74C028
:1025D000E9FF75C0EAFFEFCFFAFE0001742B000E91
:1025E0007523F34AF42AF64AF72AF75C0A0ED8B4A0
:1025F000F65CEDE3F66AF76A07EE48F0F650E92676
:10260000F750EA22EFCFFAFEF34AF42AF64AF72A05
:10261000000EF75C060ED8B4F65CEEE3F66AF76AD5
:1026200007EE3CF0F650E926F750EA22EFCFFAFE2B
:10263000F34AF42AF64AF72A000EF75C040ED8B4DF
:10264000F65CEEE3F66AF76A0AEE22F0F650E92647
:10265000F750EA22EFCFFAFEF34AF42AF64AF72AB5
:10266000000EF75C060ED8B4F65CEEE3F66AF76A85
:102670000AEE38F0F650E926F750EA22EFCFFAFEDC
:10268000F34AF42AF64AF72A000EF75C040ED8B48F
:10269000F65CEEE3F3CFE6FEF450E8CFE7FE0E0182
:1026A000FCA304D00E01FC93DF8FDF9F9E980E01E8
:1026B000DF870E01DFB7FDD7F34AF42AF3CFE0FE40
:1026C000F4CFE1FEF36AF46A07EEA2F0F350E926D4
:1026D000F450EA22FACEEFFFF34AF42A000EF45C3B
:1026E000070ED8B4F35CF0E30E01FDA31200000165
:1026F000D80EEE6F0F0E3AEF1EF0A8C7E8FF0D0AD6
:1027000028E10001150EE66F0F0EE76F400E35EC65
:1027100009F0150EE16ED96AE150D95C15E2D9CF06
:1027200000F0016A0050000FF66E0150F76E0F0EB8
:10273000F722D9500AEE52F0E926000EEA220800EC
:10274000F5CFEFFFD92AE8D70001E1CF94F0956BE0
:10275000120092C094F093C095F0120040CA8FF01E
:1027600041CA8EF02ACAE8FF0F0B040D2CCA01F0F3
:102770002DCA00F0F350005C026EF4500158036E55
:102780004ACA00F0F00E001600380F0B040DF3508B
:10279000025CE8CF92F0F4500358E8CF93F00A01BE
:1027A0004BA9A7D000018F511F0A980ED8B48E19DB
:1027B00001E09FD000019251931101E09AD0080EE0
:1027C00046CA00F0016A026A036A38EC03F000C0EE
:1027D000DAF001C0DBF002C0DCF003C0DDF047CA74
:1027E00000F0016A026A036A0001DA510026DB5137
:1027F0000122DC510222DD510322080E38EC03F0E5
:1028000000C0DEF001C0DFF002C0E0F003C0E1F084
:1028100048CA00F0016A026A036ADE510026DF51ED
:102820000122E0510222E1510322080E38EC03F0AC
:1028300000C0E2F001C0E3F002C0E4F003C0E5F044
:1028400049CA00F0E2510024E8CFAAF0000EE321CB
:10285000E8CFABF0000EE421E8CFACF0000EE521AC
:10286000E8CFADF007015EA144D007015E91AAC098
:10287000B6F0ABC0B7F0ACC0B8F0ADC0B9F0150E53
:10288000F36EE16AF350E15C15E2E1CF00F0016A1A
:102890000050000FF66E0150F76E0F0EF722E15058
:1028A0000AEE52F0E926000EEA220800F5CFEFFF0B
:1028B000E12AE8D70001F3CF94F0956B94C000F0C3
:1028C00095C001F0026A036AB6C0E8FF0024E8CFB1
:1028D000A2F0B7C0E8FF0120E8CFA3F0B8C0E8FF3E
:1028E0000220E8CFA4F0B9C0E8FF0320E8CFA5F0AC
:1028F0007CDB0A014BA9D1D000018F511F0A980E31
:10290000D8B48E1901E0C9D000019251931101E1B0
:10291000C4D00001D96B92C000F093C001F0D9C0BF
:1029200002F0036A0150035C02E10050025C13E212
:102930000001D9511AEE52F0E126000EE222D951DF
:1029400007EEA8F0E926000EEA22E7CFEFFFD5DE7A
:102950000001D92BE0D7080E46CA00F0016A026ACE
:10296000036A38EC03F000C0DAF001C0DBF002C00B
:10297000DCF003C0DDF047CA00F0016A026A036AB6
:102980000001DA510026DB510122DC510222DD5127
:102990000322080E38EC03F000C0DEF001C0DFF0C7
:1029A00002C0E0F003C0E1F048CA00F0016A026A28
:1029B000036ADE510026DF510122E0510222E1517B
:1029C0000322080E38EC03F000C0E2F001C0E3F08F
:1029D00002C0E4F003C0E5F049CA00F0E25100246F
:1029E000E8CFAAF0000EE321E8CFABF0000EE4211F
:1029F000E8CFACF0000EE521E8CFADF000EEAAF094
:102A00000001EE52EE52EE52ED50A55D08E1ED50A0
:102A1000A45D05E1ED50A35D02E1EF50A25D22E36C
:102A2000A2C000F0AA51005EA3C001F0AB51015A50
:102A3000A4C002F0AC51025AA5C003F0AD51035A34
:102A400000EEA2F00050EE5CE8CFB6F00150EE5878
:102A5000E8CFB7F00250EE58E8CFB8F00350EE5888
:102A6000E8CFB9F094C000F095C001F0026A036AA3
:102A7000B6C0E8FF0024E8CFA2F0B7C0E8FF01200D
:102A8000E8CFA3F0B8C0E8FF0220E8CFA4F0B9C0B7
:102A9000E8FF0320E8CFA5F0A8DA0A014BA336D15E
:102AA00000018F511F0A980ED8B48E1901E02ED163
:102AB0000001010E926F936B07015E8109EC1CF01F
:102AC0003ECAE1FF40CA3EFAE1CF40FA3FCAE1FF09
:102AD00041CA3FFAE1CF41FAF2D90001722B000E50
:102AE00073237251731108E0722B000E7323731D50
:102AF000FF0ED8B4721905E10001340E726F120E88
:102B0000736F100E72C000F073C001F0026A036AA6
:102B100038EC03F0FF0E0024E8CFB6F0FF0E0120E2
:102B2000E8CFB7F0000E0220E8CFB8F0000E032087
:102B3000E8CFB9F0B6C000F0B7C001F0B8C002F0FD
:102B4000B9C003F0006A016A026A180E2DEC03F0A6
:102B500000C042FAB6C000F0B7C001F0B8C002F041
:102B6000B9C003F0006A016A036A100E2DEC03F08D
:102B700000C043FAB6C000F0B7C001F0B8C002F020
:102B8000B9C003F0006A026A036A080E2DEC03F074
:102B900000C044FAB6C045FA0A014B6B4B834B891F
:102BA0000A014E6B0A014F6B00EEA6F0EE6AEE6A68
:102BB000EE6AEE6A0001080E7E6F7F6B360E746F50
:102BC0000A0E756F6FEC1CF033CAE8FF00EEA6F03A
:102BD000EE26000EEE22EE22ED22ED52ED522ACA32
:102BE000E8FF0F0B040D2CCA01F02DCA00F0F350C2
:102BF000005CE8CF96F0F4500158E8CF97F096C00B
:102C000000F097C001F000EEA6F00050EE26015053
:102C1000EE22000EEE22ED22ED52ED5296C07EF035
:102C200097C07FF000013E0E746F0A0E756F6FEC57
:102C30001CF0A6C000F0A7C001F0A8C002F0A9C017
:102C400003F0006A016A100E2DEC03F0A6C0E8FF45
:102C50000024026EA7C0E8FF0120036E021C006E74
:102C6000031C016E00C076F001C077F077C000F061
:102C7000016A00C04EFA76C04FFA0A0EF36E1A0EC1
:102C8000F46E0A0EE8CFE2FE1A0EE8CFE3FE0E0E57
:102C9000E8CFFAFEF34AF42A90C000F091C001F0A8
:102CA0000050F3260150F422F3CFE6FEF4CFE7FE06
:102CB000F60EF324F66EE50EF420F76E1C0EE16EB0
:102CC0000A0EE26EF750F61007E0E7CFFAFEE65282
:102CD000F606D8A0F706F6D7FCCE00F0020E0016D6
:102CE000000404E10E01FC93DF87DF979E980E013C
:102CF000DF87DFCE00F0080E00160004FAE00001C6
:102D0000210EEE6F100EEF6F22EC03F00A014BA1C3
:102D1000120000018F511F0A980ED8B48E19D8A442
:102D2000120000019251931122E00001D96B92C070
:102D300000F093C001F0D9C002F0036A0150035CB7
:102D400002E10050025C13E20001D9511AEE52F088
:102D5000E126000EE222D95107EEA8F0E926000E86
:102D6000EA22E7CFEFFFC9DC0001D92BE0D707014A
:102D70005E830001922B000E9323080E46CA00F0DA
:102D8000016A026A036A38EC03F000C0DAF001C09D
:102D9000DBF002C0DCF003C0DDF047CA00F0016ADE
:102DA000026A036A0001DA510026DB510122DC517C
:102DB0000222DD510322080E38EC03F000C0DEF0E1
:102DC00001C0DFF002C0E0F003C0E1F048CA00F04B
:102DD000016A026A036ADE510026DF510122E051D6
:102DE0000222E1510322080E38EC03F000C0E2F0A9
:102DF00001C0E3F002C0E4F003C0E5F049CA00F00E
:102E0000E2510024E8CFAAF0000EE321E8CFABF0B6
:102E1000000EE421E8CFACF0000EE521E8CFADF0E4
:102E200000EEAAF00001EE52EE52EE52ED50A55D1A
:102E300008E1ED50A45D05E1ED50A35D02E1EF5026
:102E4000A25D22E3A2C000F0AA51005EA3C001F07F
:102E5000AB51015AA4C002F0AC51025AA5C003F014
:102E6000AD51035A00EEA2F00050EE5CE8CFB6F090
:102E70000150EE58E8CFB7F00250EE58E8CFB8F066
:102E80000350EE58E8CFB9F094C000F095C001F0BF
:102E9000026A036AB6C0E8FF0024E8CFA2F0B7C018
:102EA000E8FF0120E8CFA3F0B8C0E8FF0220E8CF98
:102EB000A4F0B9C0E8FF0320E8CFA5F096D0080E33
:102EC00042CA00F0016A026A036A38EC03F000C0EB
:102ED000E6F001C0E7F002C0E8F003C0E9F043CA41
:102EE00000F0016A026A036A0001E6510026E75118
:102EF0000122E8510222E9510322080E38EC03F0C6
:102F000000C0EAF001C0EBF002C0ECF003C0EDF04D
:102F100044CA00F0016A026A036AEA510026EB51D2
:102F20000122EC510222ED510322080E38EC03F08D
:102F300000C0EEF001C0EFF002C0F0F003C0F1F00D
:102F400045CA00F0EE510024E8CF9EF0000EEF21BC
:102F5000E8CF9FF0000EF021E8CFA0F0000EF121A5
:102F6000E8CFA1F092C000F093C001F000EE9EF017
:102F70000050EE260150EE22000EEE22ED22ED5220
:102F8000ED529EC000F09FC001F0A0C002F0A1C0B1
:102F900003F0006A016A026A180E2DEC03F000C00B
:102FA00046FA9EC000F09FC001F0A0C002F0A1C090
:102FB00003F0006A016A036A100E2DEC03F000C0F2
:102FC00047FA9EC000F09FC001F0A0C002F0A1C06F
:102FD00003F0006A026A036A080E2DEC03F0005049
:102FE000E8CF48FA9EC049FA12000001280E942545
:102FF000E8CF80F0000E9521E8CF81F081C000F08D
:10300000016A00C02CFA80C02DFA09EC1CF03ECAFF
:10301000E1FF40CA3EFAE1CF40FA3FCAE1FF41CAB0
:103020003FFAE1CF41FA4BDFB6C000F0B7C001F084
:10303000B8C002F0B9C003F0006A016A026A180E53
:103040002DEC03F000C042FAB6C000F0B7C001F0AA
:10305000B8C002F0B9C003F0006A016A036A100E3A
:103060002DEC03F000C043FAB6C000F0B7C001F089
:10307000B8C002F0B9C003F0006A026A036A080E21
:103080002DEC03F000C044FAB6C045FA0A014B6BC0
:103090004B8907015EA304D00A014B8107015E93AF
:1030A0000A014E6B0A014F6B00EEA6F0EE6AEE6A63
:1030B000EE6AEE6A0001080E7E6F7F6B360E746F4B
:1030C0000A0E756F6FEC1CF033CAE8FF00EEA6F035
:1030D000EE26000EEE22EE22ED22ED52ED522ACA2D
:1030E000E8FF0F0B040D80C000F081C001F0F35029
:1030F000005CE8CF96F0F4500158E8CF97F096C006
:1031000000F097C001F000EEA6F00050EE2601504E
:10311000EE22000EEE22ED22ED52ED5296C07EF030
:1031200097C07FF000013E0E746F0A0E756FD7DBFB
:10313000A6C000F0A7C001F0A8C002F0A9C003F02B
:10314000006A016A100E2DEC03F0A6C0E8FF00240F
:10315000026EA7C0E8FF0120036E021C006E031C74
:10316000016E00C076F001C077F077C000F0016A10
:1031700000C04EFA76C04FFA00010E0E8025E8CF4F
:103180009AF0000E8121E8CF9BF0000E9B5D3C0E73
:10319000D8B49A5D03E23C0E9A6F9B6B0A0EF36EF5
:1031A0001A0EF46E0A0EE8CFE2FE1A0EE8CFE3FE26
:1031B0000E0EE8CFFAFEF34AF42A9AC000F09BC044
:1031C00001F00050F3260150F422F3CFE6FEF4CFD5
:1031D000E7FEF60EF324F66EE50EF420F76E1C0EF5
:1031E000E16E0A0EE26EF750F61007E0E7CFFAFE46
:1031F000E652F606D8A0F706F6D7FCCE00F0020E8F
:103200000016000404E10E01FC93DF87DF979E980F
:103210000E01DF87DFCE00F0080E00160004D8A4F0
:103220001200F8D700010A0ED86F1A0ED96F0A0ED5
:10323000E8CFE2FE1A0EE8CFE3FE0E0EE8CFFAFE6C
:10324000D84BD92B96C7B8F797C7B9F798C7BAF72D
:1032500099C7BBF79AC7BCF79BC7BDF7060ED8271F
:10326000000ED92348C7BEF749C7BFF74AC7C0F702
:103270004BC7C1F74CC7C2F74DC7C3F7060ED827D7
:10328000000ED923080EE8CFC4F70701C56B020E64
:103290000001D827000ED923450EE8CFC6F7070155
:1032A000C76B0701C86B240EE8CFC9F7040E0001F5
:1032B000D827000ED92300017C2B7D237CC0CAF7C0
:1032C0007DC000F0016A00C0CBF7020E0001D827D4
:1032D000000ED9230701CC6B0701CD6B020E000154
:1032E000D827000ED923800EE8CFCEF7110EE8CFF5
:1032F000CFF7F36AF46A07EE3CF0F350E926F45096
:10330000EA2217EED2F0F350E126F450E222EFCF9A
:10331000E7FF07EE40F0F350E926F450EA2217EEFB
:10332000D6F0F350E126F450E222EFCFE7FF020E91
:103330000001D827000ED923F34AF42AF45C040EC6
:10334000D8B4F35CD8E30701D06B0701D16B00EE72
:10335000A6F0EE6AEE6AEE6AEE6AC6C7E8FF0F0BE9
:10336000040DF3CF7EF0F4CF7FF00001C60E746F32
:10337000070E756FB4DAA6C000F0A7C001F0A8C0B0
:1033800002F0A9C003F0006A016A100E2DEC03F0F0
:10339000A6C0E8FF0024026EA7C0E8FF0120036E6C
:1033A000021C006E031C016E00C076F001C077F0B5
:1033B00077C000F0016A00C0D0F776C0D1F7040EE4
:1033C0000001D827000ED923130EE8CFDAF7880EB4
:1033D000E8CFDBF7020ED827000ED9230701DC6BFC
:1033E000070EE8CFDDF7020E0001D827000ED92323
:1033F0000701DE6B100EE8CFDFF7020E0001D827C1
:10340000000ED923020ED827000ED923F36AF46ADE
:1034100007EEE2F0F350E926F450EA22F350300FC1
:10342000EF6EF34AF42A000EF45C080ED8B4F35C95
:10343000EFE3080E0001D827000ED9230701E06B47
:103440000701E16B00EEA6F0EE6AEE6AEE6AEE6A44
:103450000001080E7E6F7F6BD20E746F070E756FC2
:103460003EDACFC7E8FF00EEA6F0EE26000EEE2211
:10347000EE22ED22ED52ED520001020E7E6F7F6BC7
:10348000DE0E746F070E756F2ADADEC77FF0DFC7B6
:103490007EF00001DA0E746F070E756F20DAA6C099
:1034A00000F0A7C001F0A8C002F0A9C003F0006AB4
:1034B000016A100E2DEC03F0A6C0E8FF0024026E96
:1034C000A7C0E8FF0120036E021C006E031C016E02
:1034D00000C076F001C077F077C000F0016A00C04C
:1034E000E0F776C0E1F7D8C0E6FE0001D9C0E7FEFC
:1034F000F60ED825F36EE50ED921F46E1C0EE16EA2
:103500000A0EE26EF450F31007E0E7CFFAFEE6523F
:10351000F306D8A0F406F6D7FCCE00F0020E001693
:10352000000404E10E01FC93DF87DF979E980E01F3
:10353000DF87DFCE00F0080E00160004FAE000017D
:10354000D84BD92BD8C0E0FED9C0E1FEF36AF46AAB
:1035500007EEA2F0F350E926F450EA22FACEEFFF8C
:10356000F34AF42A000EF45C070ED8B4F35CF0E3DF
:10357000FDCE00F0020E0016000405E10001FB0E76
:10358000EE6F0F0E77D300019C2B000E9D231200CF
:103590000AEE40F0EF50D8A4120041CAE8FF070A33
:1035A000D8A4120036D93ECAE1FF40CA3EFAE1CFA4
:1035B00040FA3FCAE1FF41CA3FFAE1CF41FA0A01AE
:1035C000446B0A01456B00EEA6F0EE6AEE6AEE6A05
:1035D000EE6A0001080E7E6F7F6B360E746F0A0E66
:1035E000756F7DD933CAE8FF00EEA6F0EE26000E17
:1035F000EE22EE22ED22ED52ED520001020E7E6F20
:103600007F6B420E746F0A0E756F69D942CA7FF0E4
:1036100043CA7EF000013E0E746F0A0E756F5FD9CB
:10362000A6C000F0A7C001F0A8C002F0A9C003F036
:10363000006A016A100E2DEC03F0A6C0E8FF00241A
:10364000026EA7C0E8FF0120036E021C006E031C7F
:10365000016E00C076F001C077F077C000F0016A1B
:1036600000C044FA76C045FA0A0EF36E1A0EF46EE4
:103670000A0EE8CFE2FE1A0EE8CFE3FE0E0EE8CF08
:10368000FAFEF34AF42A93C701F0006A92C702F0E7
:10369000FC0E0224F66EF76AFF0EF722F6500024A5
:1036A000026E000E0120036E0250F3260350F42236
:1036B000F3CFE6FEF4CFE7FE1C0EE16E0A0EE26EDB
:1036C000F450F31007E0E7CFFAFEE652F306D8A075
:1036D000F406F6D7FCCEE1FFFCCE00F0020E001699
:1036E000000404E10E01FC93DF87DF979E980E0132
:1036F000DF87DFCE00F0080E00160004D8A4120009
:10370000F8D70A013E6B0A013F6B0A01406B0A01C0
:10371000416B7FD800EEA6F0EE6AEE6AEE6AEE6AC2
:103720002ACAE8FF0F0B040D2CCA01F02DCA00F0C5
:10373000F350005CE8CF7EF0F4500158E8CF7FF002
:1037400000013E0E746F0A0E756FC9D8A6C000F056
:10375000A7C001F0A8C002F0A9C003F0006A016A86
:10376000100E2DEC03F0A6C0E8FF0024026EA7C0E7
:10377000E8FF0120036E021C006E031C016E00C0F6
:1037800076F001C077F077C000F0016A00C040FA1F
:1037900076C041FA0A0EF36E1A0EF46E0A0EE8CFE6
:1037A000E2FE1A0EE8CFE3FE0E0EE8CFFAFEF34A71
:1037B000F42A93C701F0006A92C702F0FC0E0224BB
:1037C000F66EF76AFF0EF722F6500024026E000E26
:1037D0000120036E0250F3260350F422F3CFE6FEDD
:1037E000F4CFE7FE1C0EE16E0A0EE26EF450F31009
:1037F00006E0E6CFFAFEF306D8A0F406F7D70E01EE
:10380000FCA304D00E01FC93DF8FDF9F0E01DF8746
:10381000120036CA3AFA37CA3BFA38CA3CFA39CAF1
:103820003DFA3CC736FA3DC737FA3EC738FA3FC7BC
:1038300039FA22CA1CFA23CA1DFA24CA1EFA25CA5A
:103840001FFA26CA20FA27CA21FA48C722FA49C70E
:1038500023FA4AC724FA4BC725FA4CC726FA4DC7A4
:1038600027FA0A01346B0A01356B00EEA6F0EE6A06
:10387000EE6AEE6AEE6A2ACAE8FF0F0B040DF3CF78
:103880007EF0F4CF7FF000012A0E746F0A0E756F80
:1038900026D8A6C000F0A7C001F0A8C002F0A9C0B9
:1038A00003F0006A016A100E2DEC03F0A6C0E8FFD9
:1038B0000024026EA7C0E8FF0120036E021C006E08
:1038C000031C016E00C076F001C077F077C000F0F5
:1038D000016A0050E8CF34FA76C035FA12000001D0
:1038E000000E7F5D020ED8B47E5D2AE374C0E9FF4E
:1038F00075C0EAFFEFCF58F70001742B000E752357
:1039000074C0E9FF75C0EAFFEFCF59F7742B752338
:1039100058C777F059C776F076C000F077C001F04D
:1039200000EEA6F00050EE260150EE22000EEE2230
:10393000ED22ED52ED52FE0E7E27FF0E7F23CFD7F4
:1039400000017E517F11D8B4120074C0E9FF75C028
:10395000EAFFEFCF58F70701596B58C777F059C7FF
:1039600076F076C000F077C001F000EEA6F00050CF
:10397000EE260150EE22000EEE22ED22ED52ED5227
:103980001200ACA2FED7AD6E1200AC84AC981A0E39
:10399000AF6E948E948C040EAC6E800EAB6E0701ED
:1039A000506B07014F6B0701526B0701516B9F8AE8
:1039B0009F889D8AF28CF28EAB889D98AC8AAB8EE4
:1039C0001200E9CF7FFEEACF7EFEE1CF7DFEE2CF9F
:1039D0007CFED9CF7BFEDACF7AFE9EB09DA022D0AE
:1039E000800ECF6E9E9007016B2B6BC7E8FF3C0AE1
:1039F00003E16B6B0701662B66C7E8FF3C0A04E135
:103A00000701666B0701612B61C7E8FF180A02E135
:103A10000701616B07016C2B0001AE2B000EAF2379
:103A2000B023B1239EB29DA205D09E920001822BAD
:103A3000000E83239EAA14D08E82AE50E16E070141
:103A40004F29D96ED9CF4FF750C7E8FFD96200D0C0
:103A5000D95008EE1CF0E926000EEA22E1CFEFFF74
:103A6000ACA213D051C7E8FF070152190DE052294B
:103A7000D96ED9CF52F7D95009EE1CF0E926000EC5
:103A8000EA22EF50AD6E01D09D987ACEDAFF7BCE60
:103A9000D9FF7CCEE2FF7DCEE1FF7ECEEAFF7FCE76
:103AA000E9FF11004FC7E8FF07015019FBE050295B
:103AB000D96ED9CF50F7D95008EE1CF0E926000E88
:103AC000EA22EF50006E016A1200D8000701512966
:103AD000D96ED95007015219FCE0D95009EE1CF0FB
:103AE000E926000EEA22D8C0EFFFD9CF51F79D8812
:103AF000D8C000F0D9C001F012004FC7E8FF07019D
:103B00005019000ED8A4010E1200E8CFB4FE00F048
:103B1000010EE8CFB2FE00F00E018AB1FDD70E0112
:103B2000B26B00F0B8CEE1FFB9CED9FFD950F46E38
:103B3000E150F36EF3CF00F0F4CF01F01200D900A2
:103B4000E8CFB4FE00F0D9C0B6FE00F00001DA51B3
:103B5000E8CFB7FE00F00E018AA11200FCD7400E9C
:103B6000C76E210EC66E1200FC0E926E9368570E41
:103B7000946EFB0E956E976A8E868E680E01FE8B94
:103B80000E01FDA1FDD700EE82F0EE6AEE6A0001A3
:103B9000000E835D020ED8B4825DF9E38E6A0E01D9
:103BA000DF95DF970701906B0701916B0E01E86BC2
:103BB000E96B090EE8CFECFE1A0EE8CFEDFE090E18
:103BC000E8CFEAFE1A0EE8CFEBFE0A0EE8CFE4FEDD
:103BD0001A0EE8CFE5FE0D0EE8CFA0FE00F0320E83
:103BE000E8CFA2FE00F0400EE8CFA3FE00F03F0EAB
:103BF000E8CFA9FE00F0120EE8CFA6FE00F00C0EF2
:103C0000E8CFA7FE00F0EE0EE8CFAAFE00F0050E0A
:103C1000E8CFABFE00F048C784FE00F049C785FE40
:103C200000F04AC782FE00F04BC783FE00F04CC78D
:103C300080FE00F04DC781FE00F00001100ED96F2C
:103C4000010EDA6F100E7CDF0001D96BDA6B000E0B
:103C500077DF0001720ED96F040EDA6F140E70DF79
:103C6000120EE8CFA4FE0E01DF85FB6B0001880E6B
:103C7000EE6F110EEF6F22EF03F090C7E0FE91C7D9
:103C8000E1FE900EE16E070EE26EE552F36AF46A11
:103C9000000EF45C060ED8B4F35C06E2E652F34A7A
:103CA000F42AFACEE7FFF4D793C791F092C790F0C9
:103CB0001C0EE16E0A0EE26EE55290C0F3FF91C059
:103CC000F4FFF450F31007E0E652F306D8A0F40630
:103CD000FACEE7FFF6D791C787F090C786F00001CC
:103CE0008607FF0E87231A0E875D0A0ED8B4865DFD
:103CF00004E3090E866F1A0E876F0E01FE8D86C0D3
:103D0000ECFE87C000F0016A00C0EDFE28CAE8FFA3
:103D1000080A56E129CAE8FF060A52E12BCA00F058
:103D20000004D8A412002CCAE8FF080AD8A4120084
:103D30000AEE2DF0EF50D8A412002ECAE8FF060AB2
:103D4000D8A412002FCAE8FF040AD8A412003CC766
:103D5000E8FF0A01426312003DC7E8FF0A0143631E
:103D600012003EC7E8FF0A01446312003FC7E8FFA4
:103D70000A01456312001DD0A6EF12F0F36AF46A3F
:103D80001AEE32F0F350E126F450E22207EE96F0FC
:103D9000F350E926F450EA22E7CFEFFFF34AF42A82
:103DA000000EF45C060ED8B4F35CEAE307015E870C
:103DB000120031CAE8FF010ADFE0030ADFE0120067
:103DC00028CAE8FF080A31E10AEE29F0EF502DE198
:103DD0003CC7E8FF0A013A6328D03DC7E8FF0A0163
:103DE0003B6323D03EC7E8FF0A013C631ED03FC7B8
:103DF000E8FF0A013D6319D00FD083D43ECAE8FF23
:103E0000430A02E17EEF0CF0C8EF1AF0AEEF13F0B8
:103E10008E928E948E96120033CAE8FF010AEDE06E
:103E2000070AF4E0170AEAE0F3D728CAE8FF080A0D
:103E3000D8A412000AEE29F0EF50D8A412003ACA12
:103E400000F00028D8A412003BCA00F00028D8A433
:103E500012003CCA00F00028D8A412003DCA00F0AD
:103E60000028D8A4120033CAE8FF110AD8A412000F
:103E700007015A897EEF0CF0CD90800ECF6ECE6A8E
:103E80000E0ECD6E9D800701616B0701666B070109
:103E90006B6BCD807A0ECA6E290ECB6ECA849D8262
:103EA000040EE1EC08F00001770EE66F110EE76FEB
:103EB000000E35EC09F00001CA0EE66F0F0EE76F39
:103EC000400E35EC09F061DD4FDE74EC0CF00E01B4
:103ED000D953D8A4D2DE7EEC0CF00001D8510701F2
:0C3EE0006B19F5E06BC7D8F08E78F1D7B5
:020000040001F9
:04FFF800BEFF7DFFCC
:00000001FF
